:030000000210DA11
:03000B000200A54B
:03002B000202AB23
:03005B0002040993
:030073000203E3A2
:1000800002030406080C10182030406080040608A3
:100090000C10182030406080A0C00D0D0405060D26
:1000A0000502030302C2AFC0D0C0E020620C20688A
:1000B00002419A306602415AE47385258AC262E59C
:1000C00025F470022121206802210E758B00D0E0FA
:1000D000D0D0C295C294C293D2AF32C295C294C25C
:1000E000937401D5E0FDE53C1420E21520E10D20DC
:1000F0007D02C290307D02C29202011EC2910201B5
:100100001E207D02C292307D02C29002011E758BBC
:1001100000D0E0D0D0C295C294C293D2AF32758BDA
:1001200000D0E0D0D0D2AF32419AE525600A207DE0
:1001300002D295307D02D293C294419AE5256002A5
:10014000D294207D02C293307D02C295419AE5256A
:10015000600A207D02D293307D02D295207D02C2BA
:1001600095307D02C293419A207D02D292307D0269
:10017000D290207D02D290307D02D2927401D5E0DF
:10018000FDE525600A207D02D295307D02D293C222
:1001900094419A207D02D292307D02D290D2917405
:1001A00001D5E0FDE525600A207D02D295307D0273
:1001B000D293C294419AD291207D02D292307D0294
:1001C000D2907401D5E0FDE5256002D294207D0235
:1001D000C293307D02C295419AD291207D02D29085
:1001E000307D02D2927401D5E0FDE5256002D29403
:1001F000207D02C293307D02C295419A207D02D2B9
:1002000090307D02D292D2917401D5E0FDE5256057
:100210000A207D02D293307D02D295207D02C295C4
:10022000307D02C293419A207D02D290307D02D26D
:1002300092207D02D292307D02D2907401D5E0FDF1
:10024000E525600A207D02D293307D02D295207D83
:1002500002C295307D02C293419A30723DE53C2046
:10026000E21A20E129207D02D292307D02D2902034
:100270007D02D290307D02D29202029A20E1E620E5
:100280007D02D292307D02D290D29102029AD29116
:10029000207D02D290307D02D292E525F4F58A7558
:1002A0008B00D262D0E0D0D0D2AF32C2AFC2AD5359
:1002B000E6EFC0D0C0E0D2D3D2AFC2CEE52960070E
:1002C0002074461529610978007900E580307E01A7
:1002D000F430E70278FF53DACF207E0343DA203090
:1002E0007E0343DA10C2D8C271E580307E01F4305B
:1002F000E70279FFC3E89970CE30610375291820B1
:1003000074037529188859D270E52A6004152A618A
:100310001920740543DA01C2D82070026180A859FF
:10032000206102C2702074367982B70431C3E89428
:10033000F0400374F0F8E8C4540F28F87984B70348
:1003400002615EC313C3138721200802C313200A6E
:1003500006C3C898F8615E28F8500374FFF8882235
:10036000306915E5222408F52250037522FFC3E504
:1003700022955E4003855E227882B6041885222489
:10038000A824C3E524955E4002A85EC3E8956040BA
:1003900002A8608825C3E52594404002D26420CF9E
:1003A0000CD0E0D0D0C2D343E610D2AD32C2CF7869
:1003B00001E52960053074021529C3E5599401400F
:1003C00005755C0061D7755D00756400E55C24010E
:1003D000F55C5003755CFFD0E0D0D0C2D343E6108B
:1003E000D2AD32C0D0C0E0C2AF53917F53E67FC2DE
:1003F00060759100C3E49550F594E49551F59575B9
:100400009104D0E0D0D0D2AF32C2AF53E6EFC2AD4C
:10041000C0D0C0E0C0F0D2D3D2AFA8FBA9FCC2D8F4
:10042000307102817053DACF207E0343DA10307EC0
:100430000343DA20D271E580307E01F420E70281A7
:100440004788268927C1AC53DACF207E0343DA20C0
:10045000307E0343DA10C2D8C271307402C198787A
:1004600000E580307E01F430E702C1988859C17FF1
:0F04700053DACF207E0343DA20307E0343DA10C5
:10047F00C271206102A14053DACF207E0343DA100C
:10048F00307E0343DA20C2D8D27188548955C3E82D
:10049F009552F8E99553F9E4FB7E027A00C3E8948C
:1004AF008CE994005005755800A130C3E894C8E951
:1004BF0094005008E4D2E4FB7A0AA10DC3E89468D3
:1004CF00E994015008E4D2E3FB7A0FA10DC3E8943D
:1004DF00D0E994025008E4D2E2FB7A1EA10DC3E8E2
:1004EF0094A0E994055008E4D2E1FB7A3CA10DC336
:1004FF00E89498E994085008E4D2E0FB7A787E00FB
:10050F00C3E89556FCE99557FD30E708ECF4240154
:10051F00FCEDF4FD755800C3EC9AED9E5003755831
:10052F000188568957A854A955885289537802C112
:10053F007FC3E89526F8E99527F9307C02C163302F
:10054F007B02C163307A02C15C207502A163E9FDB1
:10055F00E8FCA182E9C313F9E813F8307902C15C12
:10056F00E9C313F9E813F8307802C15CE9C313FD4E
:10057F00E813FC206126C3EC941CED94024002A109
:10058F0099ED7018C3EC94C850120528C3E5289450
:10059F000A5002C198755900D270C198E5286002BF
:1005AF0015287400207F0B7888E67896B4030278BC
:1005BF009EE624FAFEE43400FFC3EC9EFCED9FFDA3
:1005CF0092087888E6B40327A2085009207D20C23C
:1005DF00AFD27DA1EB307D17C2AFC27DC295C29461
:1005EF00C293D292D291D290206902D26BD2AFA293
:1005FF00085017E6B4030DECF42401FCEDF43400BD
:10060F00FD02061978007900C1637888E6B40315F6
:10061F00EC33FCED33FDC3EC940AFCED9400FD507C
:10062F00047C007D00C3EC94FFED9400400678FF3E
:10063F007900C163EC856FF0A4C5F0A2F733F879A8
:10064F0000400302067F78FF790002067FE9C3139B
:10065F00F9E813F8307C0EE9600278FFC3E813382D
:10066F00F8E43400F9C3E894FFE99400400278FFFE
:10067F008859D270206102C198741FF4552F4BF521
:10068F002FC274E42B7002D274752918307403755D
:10069F00290A306102C1AC20740353DAFE752A06B1
:1006AF00307403752A0AD0F0D0E0D0D0C2D3D2ADC7
:1006BF0043E6103279010206E179030206E1790A75
:1006CF000206E1791E0206E179640206E179C802A9
:1006DF0006E17817E4D5E0FDD8FAD9F6227A147B33
:1006EF00780207087A107B8C0207087A0D7BB40218
:1006FF0007087A0B7BC8020708AC2575250179021C
:10070F00B27DE4D291D5E0FDE5256002D294D5E02B
:10071F00FDC294D5E0FDC291D5E0FDE525600A202C
:10072F007D02D295307D02D293E570D5E0FD207D1C
:10073F0002C295307D02C2937496D5E0FDD9C1EA0D
:10074F00F8D5E0FDD8FBDBB1D2918C2522C37C001C
:10075F007D0075F00005F0EA33FAEB33FB50F6EB52
:10076F0013FBEA13FAC3E9FFE8FEE89AF8E99BF9ED
:10077F005004EFF9EEF8B3EC33FCED33FDD5F0DFB9
:10078F00EDF9ECF822E889F08A20D2D4F8A9F07BB1
:10079F000030F70B7BFFF42401F8E9F43400F9E89B
:1007AF008520F0A4ADF0F8E98520F0A4AFF0FEEDC0
:1007BF002EF974003FFA7C04C3EA13FAE913F9E83F
:1007CF0013F8DCF48BF030F70AE8F42401F8E9F4BD
:1007DF003400F9E889F0C2D4F8A9F0227882B6047F
:1007EF0003020848C3E5599401400302081085220B
:1007FF0024E4F53EF53FF540F541F542F547020893
:10080F00487882E6FC754701E522F523783879C7E9
:10081F00AA3AAB3BC3EB13FBEA13FAEC146013C316
:10082F00EB13FBEA13FAEC14146007C3EB13FBEAA8
:10083F0013FA12075C883E893F22E5476034C3E50F
:10084F003E9523F8E53F9400F9500CC3E89480E9F6
:10085F0094FF401602087DC3E8947FE9940050038B
:0E086F0002087D787F790002087D788079FF8D
:10087D008843894422E5476058E5432540F8E5441F
:10088D003541F9854420E4300701F43542FA30E76B
:10089D0009C3EA94F040150208BFC3EA940F500350
:1008AD000208BF78FF79FF7A0F0208BF7800790040
:1008BD007AF0C3E524955E5006E524600901D8E57C
:1008CD004420E70D01D8E54430E706884089418A88
:1008DD004222E547700302094378A1E6FAC3E543D6
:1008ED0033F8E54433F9120794E930E70BC3E89484
:1008FD0080E994FF4013211AC3E8947FE9940050D6
:10090D0002211A787F7900211A788079FFE820E793
:10091D0015C3E52398F84009C3E894014003020983
:10092D00417801020941E8F424012523F84003022E
:10093D00094178FF884522E54770030209A678A290
:10094D00E6FAA841A942120794E930E70CC3E894EE
:10095D0001E994FF401602097DC3E894FFE9940074
:10096D00500302097D78FF790002097D780179FF36
:10097D00E920E715C3E54598F84009C3E89401401F
:10098D00030209A478000209A4E8F424012545F81E
:10099D0040030209A478FF88242278FFC264E52D64
:1009AD005406702FD264C3E53B940A4009C3E52574
:1009BD0094405002C264E53B601974FF853BF0849E
:1009CD008537F0A4F8C5F0600278FFC3E895615053
:1009DD0002A8618860227883E6F520120F0075E881
:1009ED00901206C375E890E5E820ECFBA8BDA9BE02
:1009FD00120F96756B55756C00C3740013FD74550D
:100A0D0013FC74552CFC74003DFDECFAEDFBC3E8B2
:100A1D009AE99B4014E56B2455F56BE56C3400F5B4
:100A2D006CEA2CFAEB3DFB80E5AE6BAF6CC3E56C6D
:100A3D0013F9E56B13F8C3E913F9E813F8E56B281F
:100A4D00F569E56C39F56A7A03C3E913F9E813F82A
:100A5D00DAF7AA201A7009756B00756C00020A7D11
:100A6D001AEA6008EE28FEEF39FFDAF88E6B8F6C0C
:100A7D002275E890227883E6FFE5E820ECF7A8BD23
:100A8D00A9BE056DC3E56D94084052756D00E9FA78
:100A9D0079A0E76044EA7007E56E601B020AB8C3EF
:100AAD00E8956E6010E56E5006600C14020AC404E1
:100ABD0060F9020AC4E56EF56EC3946D401B755E58
:100ACD00C0C394044013755E80C39404400B755EDF
:100ADD0040C394044003755E0075BB0622EFC394BA
:100AED0001601BC3E894FFE994035012C3E8956BB2
:100AFD00E9956C5009E55E601A155E020B20E55E06
:100B0D00F46010055E7888E6B40308E55E240440C1
:100B1D0002F55EA85EC3E524985002A824C3E895AB
:100B2D005F400AA85FE55FF46003855F5E7982B779
:100B3D000402614BC3E895604002A8608825E56D0D
:100B4D00B4070375BB1022743279A387F0A4C5F0E6
:100B5D00A2F733F8C3E8955E4002A85E8822882488
:100B6D008825886122753A00753B7F2275C820A8BB
:100B7D00CCA9CD75C824AA38AB3988388939C3E8D2
:100B8D009AF8E99BF9AA3AAB3BAC3AAD3B7E047FB0
:100B9D0002C3EB940440021E1FC3EB940840021ED7
:100BAD001FC3ED13FDEC13FCDEF7C3EA9CFAEB9DBE
:100BBD00FBEF6009C3E913F9E813F8DFF7EA28FA48
:100BCD00EB39FB8A3A8B3B400122753AFF753BFFAF
:100BDD002230600261DE854C50854D51D26043E676
:100BED0080227892E6FFC3E535948240010FC3E57C
:100BFD003594A040010FC3EF940640027F057E029D
:100C0D001E3072010EC3E53B940350060E0E30727A
:100C1D00010EC3E53B940250060E0E3072010EA973
:100C2D003BA83A7A04C3E913F9E813F8DAF7C3E8F5
:100C3D009EF8E99400F94009C3E89402E994005044
:100C4D00047802E4F9E9FBE8FAC3E913FDE813FCC3
:100C5D00884C894DC3EF94036037EF20E00DE82CED
:0F0C6D00F8E93DF9ECFAEDFB020C8BE828F8E909
:100C7C0039F9C3E89402F8E99400F97A02E4FBC369
:100C8C00EF9403400D8A4E8B4F884889498C4A8DCE
:100C9C004B22884E894F8A488B498C4A8D4B223087
:100CAC00600281ABD26043E680E52D54066027A834
:100CBC003AA93BE53494085006E820E002A94D75AA
:100CCC009100C3E498F594E499F595759104D2607C
:100CDC0053917F43E68022D265753D00752000025A
:100CEC000CF6D265753D00752040E52D540660026A
:100CFC00C265D2AF206005E53D60012278017A0221
:100D0C00C3E53B940540027802C3E53B940A4002DC
:100D1C007803C3E53B940F40027A03306904781ED4
:100D2C007A01206007E53D6003D2AF22D2AF00000C
:100D3C00C2AFC3E53BFB940F40027B0FEB04307357
:100D4C00012320620123F93069027982E58BC39972
:100D5C0040D0053DEAFBE59B5440B52004DBF7A1F0
:100D6C009120650281F6C265759100AE3AAF3BC326
:100D7C00E49EF594E49FF595759104D26053917FB0
:100D8C0043E68081F630650281F6D896D2AF2230E8
:100D9C00690B0534206016753400020DB920600D06
:100DAC0020650A206B071581158102159622A84E25
:100DBC00A94F75910053917FC3E498F594E499F58C
:100DCC0095759104854850854951D26043E680223F
:100DDC0078003064053065027801E53575F007A4BC
:100DEC00F9E5F028F5F0E9A2F013A2F113A2F21341
:100DFC00F535C394785003753578C3E53595364091
:100E0C0008D266C295C294C293306002C115854A5D
:100E1C0050854B51D26043E68022C2AFD292D29120
:100E2C00D29030720B9001FC7401D5E0FD020E3CA7
:100E3C00207D02C292307D02C290759F11753C02DA
:100E4C00020F7BC2AF207D02C293307D02C295306F
:100E5C0072179001D9D291207D02D290307D02D2AE
:100E6C00927401D5E0FD020E7890013C306206E5EB
:100E7C00256002D294207D03759F01307D03759F00
:100E8C0021753C03020F7BC2AFD292D291D290302B
:100E9C00720B9001B67401D5E0FD020EA9207D0203
:100EAC00C290307D02C292207D03759F21307D035C
:100EBC00759F01753C04020F7BC2AFC29430721750
:100ECC00900193207D02D292307D02D290D2917407
:100EDC0001D5E0FD020EE690012A30620EE5256098
:100EEC000A207D02D295307D02D293759F11753CFC
:100EFC0005020F7BC2AFD292D291D29030720B907E
:100F0C0001687401D5E0FD020F16C291207D0375B6
:100F1C009F01307D03759F21753C06020F7BC2AF8C
:100F2C00207D02C295307D02C29330721F90022741
:100F3C00207D02D292307D02D290207D02D2903060
:100F4C007D02D2927401D5E0FD020F5B90014E3010
:100F5C00620EE525600A207D02D293307D02D29587
:100F6C00207D03759F21307D03759F01753C0130F9
:100F7C006B13120F967401D5E0FD7401D5E0FDC220
:100F8C0092C291C290C266D2AF22900128C295C281
:100F9C0094C293D292D291D290C262227880760976
:100FAC000876090876040876010876030876FF08A7
:100FBC00760A087601087601087601788C760108A5
:100FCC0076FF0876FF0876FF0876FF0876FF08762E
:100FDC00030876FF0876FF0876FF0876250876D09A
:100FEC000876280876500876040876FF08760208FA
:100FFC00760008767A0876FF087601227887E6FF75
:10100C00C2727888E6C394036008C27DE630E102C0
:10101C00D27DC27E7889E630E102D27EC3EF9402A3
:10102C006008758E01D27302103B758E00C273225C
:10103C007880E6149000809378A1F67881E614907D
:10104C0000809378A2F6120F96227886E614900010
:10105C008D9378A3F6120F962222789CE67536FFB4
:0F106C0075370CB402067536A075370AB4030643
:10107B0075368275370522227896E6FA7897E6FB65
:10108B00307F047A007BFFC3EB9AFCC3948250023F
:10109B007C82756F00056FEC856FF0A4C3E5F0944F
:1010AB008040F222D27F11831206D27A007B007C21
:1010BB00101206C8E5592AFA74003BFBDCF37C04DA
:1010CB00C3EB13FBEA13FADCF7FEC27F118322E5B5
:1010DB00EF20E6037520000520903FFFE52014600C
:1010EB0006901DFF1460009304600375EF12C2D3CA
:1010FB0053D9BF7581C043FF801206C375EF0243FE
:10110B00B203E5B3240420E702F5B3120F96758002
:10111B00FF75A40075F19075D47F75908775A5BF89
:10112B0075F2BF75D50075A60175E241120FA812B5
:10113B0015C778988670C2AF1206DC1206EC120641
:10114B00D21206F31206D21206FA1206D2C2AFE47C
:10115B00F8F6D8FD78C879C8308707D9FBD8F702DD
:10116B001C00120FA81215C71108113C115611655E
:10117B0011661182118378988670120F96758850BC
:10118B0075891275C82475910475D84075A8227598
:10119B00B80275E690759B80759D0075D10E75BC78
:1011AB005875BB0675BA1175E8801206C3D2AF121B
:1011BB0009E343DA01C2D8C2711206DC753001D2E1
:1011CB00617B037A0CE55870067A0CDB022158120E
:1011DB0006D22070022158C270E559C3940240E335
:1011EB00E52F541F855B5AF55BB55AD7DAD7C26129
:1011FB0053DACF207E0343DA20307E0343DA10C26A
:10120B00D8C271C2757528001206D7307409C3E5B0
:10121B0028940A4002D2751206C8780230740278FC
:10122B0000C3E5599840F0C2AF1206EC1206EC125F
:10123B0006ECD2AF1206DC7546007888E6B40302E2
:10124B0061211206C8788CE6C39401500302132166
:10125B00E530C394015003021321207435C3E559C3
:10126B0094FF5003021321C2AF120701D2AF120633
:10127B00D7C3E559940150EFC2AF1206EC1206CD5D
:10128B001206ECD2AF1206D7C3E55994FF40E90220
:10129B00176F7F02D27F11831206D7C2AFC27F11A5
:1012AB0083AE59C3E559947FD2AF40741206C3C2C3
:1012BB00AF120701D2AFDFDC11AFC3EE9405789705
:1012CB00F61206DC1216091216F27F0AD27F118370
:1012DB001206D7C2AFC27F1183AE59C3E559947FB3
:1012EB00D2AF50E61206C3C2AF1206EC1206CD12F5
:1012FB0006ECD2AFDFD611AFEE24057896F61206C8
:10130B00DC1216091217211206D71183C3E5599463
:10131B00FF40F402176FC3E55995464003855946C4
:10132B001206D778017988E7B403027805C3E5592B
:10133B009840024145C2AF12070112070112070183
:10134B00D2AF1206DC753000E4F531F5320531E52C
:10135B0031F470390532789AE678191460127832C4
:10136B0014600D787D14600878FA146003753200F0
:10137B00C3E53298401715327531B478998670C22F
:10138B00AF120701D2AF789886701206D71206CD2E
:10139B00E529700530740221587801207402780613
:1013AB00C3E5599840A77888E6C3940360031206F7
:1013BB00D7E52970022158C2AF120F96E4F522F53A
:1013CB0023F524F525D2AF78858662F53EF53FF5FA
:1013DB0040F541F542F56DF547F52CF52DF5351238
:1013EB000B72756D0875BB101206C3120A7EE5E809
:1013FB0020ECFBA8BDA9BEE97001F8886E120A8229
:10140B00756D0875BB107887E6FE76021108788734
:10141B00EEF6C2AF755EFF120B5485225E85225F1E
:10142B00852260D2AF752201752401752501855D7A
:10143B0064756501D268D269753400120F00120F02
:10144B002A120B72120B79120BEF021463120F9606
:10145B001108756D0075BB06120CEE120D9B120D6B
:0D146B00BA1207EB120DDC120E26120B79DF
:10147800120BDE120BEF120CAB120CE3120D9B12C7
:101488000DBA1208491209A7120DDC120E4F120BE1
:1014980079120BDE120BEF120CAB120CEE120D9B35
:1014A800120DBA120882120DDC120E93120B791269
:1014B8000BDE120BEF120CAB120CE3120D9B120D8C
:1014C800BA1208DF120DDC120EC5120B79120BDEF0
:1014D800120BEF120CAB120CEE120D9B120DBA127E
:1014E8000944120DDC120F00120B79120BDE120BDD
:1014F800EF120CAB120CE3120A7E120D9B120DBAFE
:10150800120A82120DDC120F2A120B79120BDE124C
:101518000BEF120CAB306938206B3585615E856145
:101528005F855D6475650179327A0AC3E53499404F
:1015380012C269D26A8A3385615E755FFF75602061
:10154800021558C3E5599401400302146302159625
:10155800306A1E206B1BE533147007C26A755EFF84
:101568008158F533C3E55994014003021463021509
:1015780096C3E55C94FA5016307404E529600FC3ED
:10158800E53B78F0306B0278609850028163C2AF17
:10159800120F967887E6FE760211087887EEF6E451
:1015A800F522F523F524F525F562C268D2AF1206B7
:1015B800C3120F96307406E52970022158615390C2
:1015C8001A0D782012164BE520B4550CA312164BB1
:1015D800E520B4AA030215E9120FA812160902168B
:1015E80008901A0378807B0A12164BA308DBF9903F
:1015F8001A0F788C7B1512164BA308DBF9901A2466
:1016080022C2AF12168A121664901A00740D1216AE
:1016180050A37402121650A37413121650901A0392
:1016280078807B0A12164FA308DBF9901A0F788C82
:101638007B1512164FA308DBF912169D12167B9024
:101648001A2422E493F622E6438F01538FFD75EFA7
:101658000275B7A575B7F1F0538FFE22438F024389
:101668008F0175EF0275B7A575B7F1901A0DF05394
:101678008FFC22901A0D7455D150901A0E74AAD16D
:1016880050227A3079D07820901A40D14BE520F753
:1016980009A3DAF7227A3079D0901A40E7D15009B5
:1016A800A3DAF922AB71A872BB01027980BB0202EE
:1016B8007981BB03027982BB04027984BB05027974
:1016C80083BB06027986BB07027992BB0802798739
:1016D800BB0902799CBB0A027988BB0B027989E8AD
:1016E800F7227C051206DCDCFB22C2AF1206EC12E4
:1016F80006F31206FA1207011206CD1206EC1206BC
:10170800F31206FA1207011206CD1206EC1206F3BE
:101718001206FA120701D2AF22C2AF12070112064F
:10172800FA1206F31206EC1206CD1207011206FA97
:101738001206F31206EC1206CD1207011206FA126F
:1017480006F31206ECD2AF22AE71AF72C2AF120628
:10175800EC1206EC1206EC1206CDDEF212070112AC
:1017680006CDDFF8D2AF22D1F2D1EAD1EA75710104
:10177800757201757300F1507C05AD591206DCC312
:10178800ED955970F5C3E5599401400AC3E559949C
:10179800FF40320217ABD1ACD109D1F2C2AF75EF1D
:1017A80012D1EADCD50573C3E5739403500280C6F1
:1017B800D1EA0572E5711490009A93F808C3E572AE
:1017C80098500280AED1EAD1EA0571C3E571940C54
:1017D8005002809C120FA8D109C2AF75EF12D1EA4E
:101A00000D02130909040103FF0A01010155AA018E
:101A1000FFFFFFFFFF03FFFFFF25D0285004FF0259
:051A2000007AFF01FF48
:101A400023585032354123202020202020202020E0
:101A500023424C48454C4923463333302320202031
:101A60002020202020202020202020202020202076
:101C0000C2AFC2D353D9BF7581C043B20343FF8073
:101C1000752438752503B1BF75EF0275E24043F1B5
:101C20008053A47FD287780379E67C1075220075F3
:101C30002300901DCC7B0675249875250130870202
:101C4000813D208708D8FBD9F9DCF781AD308708C2
:101C5000D8FBD9F9DCF781ADB17FE493A3C39A60D7
:101C6000028126DBDDB171600281267B08E493FAF4
:101C7000A3B152DBF87A30B152752200752300B15E
:101C800071EAFCEBFDC3ED94FE400EB1718A278B27
:101C900028ED30E0048A828B83B1717AC270D8C398
:101CA000ED94FE601050CEBD0022EC600675200061
:101CB0000200008100A827A9280809D804D90281B8
:101CC000C9B175EA89AAF281BB0D8199C3ED94036C
:101CD0005049EDA2E092007AC5C3E5829400E58305
:101CE000941C5093200010438F02438F0175B7A5B9
:101CF00075B7F1F030001FA827A9280809438F0104
:101D0000538FFDD804D902A11689AAE275B7A5752B
:101D1000B7F1F0A3A103538FFC81757AC1BD030C09
:101D2000E493A3FAB136DCF8B12E81758177AA224B
:101D3000AB23B152EBFAEA6222752608C3E52313FE
:101D4000F523E52213F52250066323A0632201D573
:101D500026EAB1BFB1BF75260AEAF4200102D28794
:101D6000300102C287B1BFC3134002C201D526EBC6
:101D700022B175EAFB208702A175308702A17A752E
:101D80002608AE24AF25C3EF13FFEE13FEB1C3B197
:101D9000BFC3EA133087024480FA30E703632201AD
:101DA000C3E52313F523E52213F52250066323A090
:101DB000632201D526D9E52265236523F52222AECB
:101DC00024AF250E0FDEFEDFFCD20122424C486517
:0A1DD0006C6934373132F33006013C
:00000001FF
